:020000040000FA
:02000000752861
:08000800F100030EF000831665
:1000100003138C1E0F28831203138C1A18288316BF
:1000200003130C1E1728831203130C1A2728702899
:10003000831203131A08F200743072020319761443
:1000400083120313981C0F28181218160F287B18F8
:100050005428761C172876100508F4000608F500C9
:100060000730F405F830F50574087504F300F9015C
:10007000F801F701F30AF30B45283030F704F804D0
:10008000F9040530FA007B145428F70AF70A0A30FD
:100090007702031D3B28F701F80A0A307802031D96
:1000A0003B28F801F90A3B2883120313FA0B5A285C
:1000B0007B10172804307A02031D602879086E2807
:1000C00003307A02031D662878086E2802307A020F
:1000D000031D6C282C306E2877086E28990017288D
:1000E000700E8300F10E710E090083120313850157
:1000F000860107309F0083160313FF308500FF3011
:100100008600193099002430980083120313903030
:100110009800F201F301F601FB01831603138B171C
:0E0120000B178C160C168312031396289628C4
:02400E00223F4F
:00000001FF
